
 pwfolder

 Start         Length     Name                   Class
 0001:00000000 000003F5CH CODE32                 CODE 32-bit
 0002:00000000 000000019H CODE16                 CODE 16-bit
 0003:00000000 000000030H _MSGSEG32              CODE 32-bit
 0004:00000000 000001468H DATA32                 DATA 32-bit
 0004:00001468 000000154H CONST32                CONST 32-bit
 0004:000015BC 000000000H BSS32                  BSS 32-bit
 0004:000015BC 0000000D0H c_common               BSS 32-bit
 0005:00000000 00000000CH EDC1                   EDC_CLASS 32-bit
 0005:0000000C 000000138H EDC2                   EDC_CLASS 32-bit
 0005:00000144 000000004H EDC3                   EDC_CLASS 32-bit
 0006:00000000 000000000H STACK32                STACK 32-bit
 0006:00000000 000000008H ASMD16                 DATA16 16-bit

 Origin   Group
 0004:0   DGROUP
 0005:0   _EIBGROUP
 0000:0   FLAT

 Address       Export                  Alias

 0004:00000020 M_PWFolderCClassData    M_PWFolderCClassData
 0004:0000001C M_PWFolderClassData     M_PWFolderClassData
 0001:000008F4 M_PWFolderNewClass      M_PWFolderNewClass
 0004:00000014 PWFolderCClassData      PWFolderCClassData
 0004:00000004 PWFolderClassData       PWFolderClassData
 0001:00000504 PWFolderNewClass        PWFolderNewClass

  Address         Publics by Name

 0004:000015F4       @BSSEDCINIT.C
 0004:000015C0       @BSSN_EXCEPT.C
 0004:0000167C       @BSSPRTEMSG.C
 0004:00001664       @BSSpwfolder.c
 0004:00000000       DefaultClassTitle
 0000:00000000  Imp  DOS32FLATTOSEL       (DOSCALLS.425)
 0003:00000012       DOS32GETMESSAGE
 0003:00000012       Dos32GetMessage
 0000:00000000  Imp  DOS32IQUERYMESSAGECP (MSG.8)
 0000:00000000  Imp  DOS32SELTOFLAT       (DOSCALLS.426)
 0000:00000000  Imp  DOS32TRUEGETMESSAGE  (MSG.6)
 0000:00000000  Imp  DosAllocMem          (DOSCALLS.299)
 0000:00000000  Imp  DosCreateMutexSem    (DOSCALLS.331)
 0000:00000000  Imp  DosExit              (DOSCALLS.234)
 0000:00000000  Imp  DosFreeMem           (DOSCALLS.304)
 0000:00000000  Imp  DosFreeModule        (DOSCALLS.322)
 0000:00000000  Imp  DosGetInfoBlocks     (DOSCALLS.312)
 0003:00000012       DOSGETMESSAGE
 0003:00000012       DosGetMessage
 0000:00000000  Imp  DosLoadModule        (DOSCALLS.318)
 0000:00000000  Imp  DosQueryDBCSEnv      (NLS.6)
 0000:00000000  Imp  DosQueryHType        (DOSCALLS.224)
 0000:00000000  Imp  DosQuerySysInfo      (DOSCALLS.348)
 0000:00000000  Imp  DosRaiseException    (DOSCALLS.356)
 0000:00000000  Imp  DosReleaseMutexSem   (DOSCALLS.335)
 0000:00000000  Imp  DosRequestMutexSem   (DOSCALLS.334)
 0000:00000000  Imp  DosSetFilePtr        (DOSCALLS.256)
 0000:00000000  Imp  DosSetSignalExceptionFocus (DOSCALLS.378)
 0000:00000000  Imp  DosWrite             (DOSCALLS.282)
 0004:0000160C       errno
 0001:000036F0       fflush
 0001:00001990       free
 0001:00003848       getenv
 0004:000015F0       hLockedIcon
 0004:0000165C       hmodThisClass
 0004:00001658       hUnlockedIcon
 0001:00001A34       malloc
 0004:00000020       M_PWFolderCClassData
 0004:0000001C       M_PWFolderClassData
 0001:000008F4       M_PWFolderNewClass
 0000:00000000  Imp  M_WPFolderNewClass   (PMWP.315)
 0000:00000000  Imp  M_WPObjectClassData  (PMWP.323)
 0001:00001718       PasswordDlgProc
 0004:00000014       PWFolderCClassData
 0004:00000004       PWFolderClassData
 0001:000015FC       pwfoldercls_wpclsInitData
 0001:000015A8       pwfoldercls_wpclsQueryIcon
 0001:00001568       pwfoldercls_wpclsQueryTitle
 0001:0000169C       pwfoldercls_wpclsUnInitData
 0001:00000504       PWFolderNewClass
 0001:00000B4C       pwfolder_LockFolder
 0001:00000A44       pwfolder_QueryInfo
 0001:00000AC8       pwfolder_SetInfo
 0001:00000C9C       pwfolder_wpInitData
 0001:00000DEC       pwfolder_wpMenuItemSelected
 0001:00000D28       pwfolder_wpModifyPopupMenu
 0001:00000EB8       pwfolder_wpOpen
 0001:00001358       pwfolder_wpRestoreState
 0001:00001264       pwfolder_wpSaveState
 0001:000014B0       pwfolder_wpSetIcon
 0001:000010C0       pwfolder_wpSetTitle
 0001:00001174       pwfolder_wpSetup
 0003:00000000       sig32
 0000:00000000  Imp  SOMClassClassData    (som.3)
 0000:00000000  Imp  SOMClassMgrClassData (som.6)
 0000:00000000  Imp  SOMClassMgrObject    (som.7)
 0000:00000000  Imp  somConstructClass    (som.28)
 0000:00000000  Imp  somDataResolve       (som.47)
 0000:00000000  Imp  somEnvironmentNew    (som.30)
 0000:00000000  Imp  SOMError             (som.9)
 0000:00000000  Imp  somIdFromString      (som.31)
 0000:00000000  Imp  SOMObjectCClassData  (som.13)
 0000:00000000  Imp  somParentResolve     (som.33)
 0000:00000000  Imp  somPrintf            (som.35)
 0000:00000000  Imp  somResolve           (som.37)
 0000:00000000  Imp  somTestCls           (som.42)
 0000:00000000  Imp  SOM_TraceLevel       (som.18)
 0004:00000D68       stderr
 0004:00000D60       stdin
 0004:00000D64       stdout
 0001:00001D5C       strcat
 0001:00001DA0       strcmp
 0001:00001DD4       strcpy
 0001:00001E10       strlen
 0001:00003A28       strspn
 0001:00001E34       strstr
 0001:00003634       strupr
 0000:00000000  Imp  WinDefDlgProc        (PMWIN.910)
 0000:00000000  Imp  WinDestroyPointer    (PMWIN.727)
 0000:00000000  Imp  WinDismissDlg        (PMWIN.729)
 0000:00000000  Imp  WinDlgBox            (PMWIN.923)
 0000:00000000  Imp  WinLoadPointer       (PMWIN.780)
 0000:00000000  Imp  WinMessageBox        (PMWIN.789)
 0000:00000000  Imp  WinQueryDlgItemText  (PMWIN.815)
 0000:00000000  Imp  WinQueryWindowULong  (PMWIN.843)
 0000:00000000  Imp  WinSetWindowULong    (PMWIN.878)
 0000:00000000  Imp  WPFolderNewClass     (PMWP.15)
 0000:00000000  Imp  WPObjectClassData    (PMWP.23)
 0004:000015D4       _Async_exception_flag
 0001:00003388       _bisex_callback
 0001:000036A4       _bit_test_set
 0004:000015D0       _broken_time_ptr
 0001:00002A40       _critlib_except
 0001:00002D88       _CRT_init
 0001:0000321C       _CRT_term
 0004:00000D70       _ctable
 0004:000015E0       _ctype
 0004:000015E4       _cvt_buf_ptr
 0004:00000E74       _daylight
 0004:00000BF4       _dllentry
 0001:00002D48       _DLL_InitTerm
 0004:00001680       _doserrno
 0001:00001D54       _DosFlatToSel
 0001:00001D4C       _DosSelToFlat
 0004:00001608       _dttm_ptr
 0001:000036B8       _edcGetMessage
 0004:000015BC       _environ
 0001:00003364       _Exception
 0001:00001FA0       _exception_dllinit
 0001:00001F6C       _exception_procinit
 0001:00002C58       _EXE_Exception
 0001:000036DC       _fcloseall_weak
 0005:00000000       _firsteib
 0004:00001688       _flags
 0001:00003A64       _Flush
 0001:00003C14       _flushb
 0001:00003780       _FreeFCB
 0001:000033A0       _get_seglim
 0001:00001EF8       _ilog2
 0004:00001684       _internal_buf_ptr
 0005:00000144       _lasteib
 0004:00001604       _lcvt_buf_ptr
 0001:000028D8       _Lib_excpt
 0001:000032B8       _ltoa
 0001:00003350       _matherr
 0004:00000BF8       _matherr_ptr
 0001:00003208       _Math_Exception_Def
 0001:000033DC       _MesgServ
 0001:00001F00       _mig_eib_store
 0004:000015DC       _osmajor
 0004:000015EC       _osminor
 0004:00000E7C       _osmode
 0004:00001610       _pBucketArr
 0004:00001674       _perror_msg_ptr
 0004:00000D6C       _PGLOBAL_PTR
 0001:000035D0       _PrintErrMsg
 0004:00000E84       _random_seed
 0001:00002B54       _recreate_exception
 0001:00003394       _Regen_exception
 0004:000015E8       _Saved_Return_Address
 0001:00003948       _setupenv
 0004:00001678       _strerror_msg_ptr
 0004:00001660       _strtok_pos
 0004:000015D8       _tempname_ptr
 0001:00003684       _terminate
 0001:0000337C       _Test_and_reset
 0001:000031AC       _test_handle
 0004:00000E78       _timezone
 0004:0000166C       _tzname
 0004:00000E80       _version
 0001:0000362C       _w_raise
 0001:0000188C       __EDC3216
 0001:00001924       __EDCThunkProlog
 0001:00001FD0       __Exception
 0006:00000000       __fac

  Address         Publics by Value

 0000:00000000  Imp  DosExit              (DOSCALLS.234)
 0000:00000000  Imp  DOS32SELTOFLAT       (DOSCALLS.426)
 0000:00000000  Imp  WinSetWindowULong    (PMWIN.878)
 0000:00000000  Imp  SOMClassMgrClassData (som.6)
 0000:00000000  Imp  somPrintf            (som.35)
 0000:00000000  Imp  somDataResolve       (som.47)
 0000:00000000  Imp  SOMClassClassData    (som.3)
 0000:00000000  Imp  SOMError             (som.9)
 0000:00000000  Imp  somResolve           (som.37)
 0000:00000000  Imp  SOM_TraceLevel       (som.18)
 0000:00000000  Imp  WinQueryWindowULong  (PMWIN.843)
 0000:00000000  Imp  DosSetFilePtr        (DOSCALLS.256)
 0000:00000000  Imp  WinMessageBox        (PMWIN.789)
 0000:00000000  Imp  WinDestroyPointer    (PMWIN.727)
 0000:00000000  Imp  DosFreeMem           (DOSCALLS.304)
 0000:00000000  Imp  DosQueryHType        (DOSCALLS.224)
 0000:00000000  Imp  DosRequestMutexSem   (DOSCALLS.334)
 0000:00000000  Imp  somEnvironmentNew    (som.30)
 0000:00000000  Imp  WPFolderNewClass     (PMWP.15)
 0000:00000000  Imp  somParentResolve     (som.33)
 0000:00000000  Imp  WinDefDlgProc        (PMWIN.910)
 0000:00000000  Imp  WinDlgBox            (PMWIN.923)
 0000:00000000  Imp  DosQuerySysInfo      (DOSCALLS.348)
 0000:00000000  Imp  DosGetInfoBlocks     (DOSCALLS.312)
 0000:00000000  Imp  somTestCls           (som.42)
 0000:00000000  Imp  DosAllocMem          (DOSCALLS.299)
 0000:00000000  Imp  DosFreeModule        (DOSCALLS.322)
 0000:00000000  Imp  M_WPFolderNewClass   (PMWP.315)
 0000:00000000  Imp  DosSetSignalExceptionFocus (DOSCALLS.378)
 0000:00000000  Imp  DosRaiseException    (DOSCALLS.356)
 0000:00000000  Imp  M_WPObjectClassData  (PMWP.323)
 0000:00000000  Imp  DosReleaseMutexSem   (DOSCALLS.335)
 0000:00000000  Imp  DosWrite             (DOSCALLS.282)
 0000:00000000  Imp  DOS32TRUEGETMESSAGE  (MSG.6)
 0000:00000000  Imp  WinQueryDlgItemText  (PMWIN.815)
 0000:00000000  Imp  WinLoadPointer       (PMWIN.780)
 0000:00000000  Imp  DosLoadModule        (DOSCALLS.318)
 0000:00000000  Imp  DOS32IQUERYMESSAGECP (MSG.8)
 0000:00000000  Imp  DosQueryDBCSEnv      (NLS.6)
 0000:00000000  Imp  WPObjectClassData    (PMWP.23)
 0000:00000000  Imp  DOS32FLATTOSEL       (DOSCALLS.425)
 0000:00000000  Imp  somIdFromString      (som.31)
 0000:00000000  Imp  SOMClassMgrObject    (som.7)
 0000:00000000  Imp  WinDismissDlg        (PMWIN.729)
 0000:00000000  Imp  SOMObjectCClassData  (som.13)
 0000:00000000  Imp  somConstructClass    (som.28)
 0000:00000000  Imp  DosCreateMutexSem    (DOSCALLS.331)
 0001:00000504       PWFolderNewClass
 0001:000008F4       M_PWFolderNewClass
 0001:00000A44       pwfolder_QueryInfo
 0001:00000AC8       pwfolder_SetInfo
 0001:00000B4C       pwfolder_LockFolder
 0001:00000C9C       pwfolder_wpInitData
 0001:00000D28       pwfolder_wpModifyPopupMenu
 0001:00000DEC       pwfolder_wpMenuItemSelected
 0001:00000EB8       pwfolder_wpOpen
 0001:000010C0       pwfolder_wpSetTitle
 0001:00001174       pwfolder_wpSetup
 0001:00001264       pwfolder_wpSaveState
 0001:00001358       pwfolder_wpRestoreState
 0001:000014B0       pwfolder_wpSetIcon
 0001:00001568       pwfoldercls_wpclsQueryTitle
 0001:000015A8       pwfoldercls_wpclsQueryIcon
 0001:000015FC       pwfoldercls_wpclsInitData
 0001:0000169C       pwfoldercls_wpclsUnInitData
 0001:00001718       PasswordDlgProc
 0001:0000188C       __EDC3216
 0001:00001924       __EDCThunkProlog
 0001:00001990       free
 0001:00001A34       malloc
 0001:00001D4C       _DosSelToFlat
 0001:00001D54       _DosFlatToSel
 0001:00001D5C       strcat
 0001:00001DA0       strcmp
 0001:00001DD4       strcpy
 0001:00001E10       strlen
 0001:00001E34       strstr
 0001:00001EF8       _ilog2
 0001:00001F00       _mig_eib_store
 0001:00001F6C       _exception_procinit
 0001:00001FA0       _exception_dllinit
 0001:00001FD0       __Exception
 0001:000028D8       _Lib_excpt
 0001:00002A40       _critlib_except
 0001:00002B54       _recreate_exception
 0001:00002C58       _EXE_Exception
 0001:00002D48       _DLL_InitTerm
 0001:00002D88       _CRT_init
 0001:000031AC       _test_handle
 0001:00003208       _Math_Exception_Def
 0001:0000321C       _CRT_term
 0001:000032B8       _ltoa
 0001:00003350       _matherr
 0001:00003364       _Exception
 0001:0000337C       _Test_and_reset
 0001:00003388       _bisex_callback
 0001:00003394       _Regen_exception
 0001:000033A0       _get_seglim
 0001:000033DC       _MesgServ
 0001:000035D0       _PrintErrMsg
 0001:0000362C       _w_raise
 0001:00003634       strupr
 0001:00003684       _terminate
 0001:000036A4       _bit_test_set
 0001:000036B8       _edcGetMessage
 0001:000036DC       _fcloseall_weak
 0001:000036F0       fflush
 0001:00003780       _FreeFCB
 0001:00003848       getenv
 0001:00003948       _setupenv
 0001:00003A28       strspn
 0001:00003A64       _Flush
 0001:00003C14       _flushb
 0003:00000000       sig32
 0003:00000012       DOS32GETMESSAGE
 0003:00000012       Dos32GetMessage
 0003:00000012       DosGetMessage
 0003:00000012       DOSGETMESSAGE
 0004:00000000       DefaultClassTitle
 0004:00000004       PWFolderClassData
 0004:00000014       PWFolderCClassData
 0004:0000001C       M_PWFolderClassData
 0004:00000020       M_PWFolderCClassData
 0004:00000BF4       _dllentry
 0004:00000BF8       _matherr_ptr
 0004:00000D60       stdin
 0004:00000D64       stdout
 0004:00000D68       stderr
 0004:00000D6C       _PGLOBAL_PTR
 0004:00000D70       _ctable
 0004:00000E74       _daylight
 0004:00000E78       _timezone
 0004:00000E7C       _osmode
 0004:00000E80       _version
 0004:00000E84       _random_seed
 0004:000015BC       _environ
 0004:000015C0       @BSSN_EXCEPT.C
 0004:000015D0       _broken_time_ptr
 0004:000015D4       _Async_exception_flag
 0004:000015D8       _tempname_ptr
 0004:000015DC       _osmajor
 0004:000015E0       _ctype
 0004:000015E4       _cvt_buf_ptr
 0004:000015E8       _Saved_Return_Address
 0004:000015EC       _osminor
 0004:000015F0       hLockedIcon
 0004:000015F4       @BSSEDCINIT.C
 0004:00001604       _lcvt_buf_ptr
 0004:00001608       _dttm_ptr
 0004:0000160C       errno
 0004:00001610       _pBucketArr
 0004:00001658       hUnlockedIcon
 0004:0000165C       hmodThisClass
 0004:00001660       _strtok_pos
 0004:00001664       @BSSpwfolder.c
 0004:0000166C       _tzname
 0004:00001674       _perror_msg_ptr
 0004:00001678       _strerror_msg_ptr
 0004:0000167C       @BSSPRTEMSG.C
 0004:00001680       _doserrno
 0004:00001684       _internal_buf_ptr
 0004:00001688       _flags
 0005:00000000       _firsteib
 0005:00000144       _lasteib
 0006:00000000       __fac

Program entry point at 0001:2D48
